:102F00000C94AA170C94C5170C94C5170C94C517EC
:102F10000C94C5170C94C5170C94C5170C94C517C1
:102F20000C94C5170C94C5170C94C5170C94C517B1
:102F30000C94C5170C94C5170C94C5170C94C517A1
:102F40000C94C5170C94C5170C94C5170C94C51791
:102F50000C94C51711241FBECFE5D4E0DEBFCDBF52
:102F600010E0A0E6B0E0E0E6F7E302C005900D92C5
:102F7000A036B107D9F711E0A0E6B0E001C01D927C
:102F8000AE32B107E1F70C94021C0C948017F4C028
:102F90001FEF12BB1FEF18BB089512E011BB1AEA16
:102FA00017BB089512E011BB18E017BB0895552315
:102FB00012F0C19A01C0C1980895552312F0C1982A
:102FC00001C0C19A0895C79A13E11A95F1F7C798FD
:102FD0001AE01A95F1F7089507E109B908E10AB96D
:102FE00008955F9BFECF4CB108955D9BFECF4CB919
:102FF0000895C895002021F0402DF7DF3196F9CFD4
:103000000895C895002021F0402DEFDF3296F9CFCA
:103010000895C895002021F0501519F03296F9CF87
:1030200008940895C895002041F0501511F032968B
:10303000F9CF3196C895C02C8C2C0895C8950020E6
:1030400039F0501511F03296F9CF3196C895D02C41
:10305000089518E224E72A95F1F71A95D9F70A9509
:10306000C1F7089519D03D2F17D03C2F15D00895E2
:10307000312D12D0322D10D0332D0ED0342F0CD054
:103080000895312D09D0322D07D0332D05D003D02E
:10309000432FABDF0895332708E070E0331F10F4AF
:1030A000C59A01C0C598770FB69971608CDF0A95F3
:1030B000A9F7372F0895552322F030E2EDDF3D2F99
:1030C00003C03D2F41D03160E7DF3C2FE5DFE3DF78
:1030D000432F8BDF55234AF038E2DEDF3D2FDCDF64
:1030E0003C2FDADFD8DF432F80DF21960895552368
:1030F00022F030EAD1DF3D2F05C0573859F03D2F7F
:1031000023D03560C9DF3C2FC7DFC5DF432F6DDF1C
:10311000219608950F910F91A2C2552322F030EC11
:10312000BBDF3D2F05C0573861F03D2F0DD0366015
:10313000B3DF3C2FB1DF342FAFDF0AE08ADF219607
:1031400008950F910F918BC2330F330F330F18F483
:10315000573809F434600895C39808EC7ADF08EC16
:1031600078DF38ECC39A02E074DFC39801E071DFC6
:103170003A95C1F7C39A089500E1C02E8C2C50E215
:10318000AA24992405DF0EDF27DFE6DF2ADF4B3193
:10319000E9F3443579F425DF542FE5E4FBE1EE0F44
:1031A000FF1F40DF0FEFD02EE5E3FBE1EE0FFF1F27
:1031B00045DF58C2433531F4E9E7FBE1EE0FFF1F6D
:1031C00018DFE4CF463531F4E5E7FBE1EE0FFF1FF2
:1031D00010DFDCCF463731F4E7E7FBE1EE0FFF1FEE
:1031E00008DFD4CF443769F4E5E3FBE1EE0FFF1FBE
:1031F00008DFE5E4FBE1EE0FFF1F03DF40E0F5DE53
:10320000C5CF403719F443E5F0DEC0CF413619F49D
:1032100049E5EBDEBBCF493641F4EDE7FBE1EE0FCC
:10322000FF1FE7DE4AE0E1DE1DC2423639F449E520
:10323000DCDE40E0DADE40E2D8DEA8CF483719F421
:10324000D0DEC39A0FC2493719F4CBDEC3980AC245
:10325000E5E3FBE1EE0FFF1FDCDE38F4E5E4FBE124
:10326000EE0FFF1FD6DE08F4FAC1403509F028C082
:10327000C39893DEC7989BDE02E3EBDE9EDE02E39B
:10328000E8DE3CEA09DF33E507DF503280F0552302
:1032900072F020E200DF333561F030E0FDDE93DED6
:1032A0003CEAFADE33E5F8DE2A95A1F702C030E009
:1032B000F3DE552312F030E0EFDE04E0CADED2C1C7
:1032C0004336B9F48EDE30E4832F55231AF0E4DE62
:1032D0003D2F03C03D2F38DF3260DEDE3C2FDCDEC9
:1032E000342FDADE942F4C2E5D2E55230AF42196CE
:1032F0005DC1433491F475DE552372F038E4832FB9
:10330000CBDE3D2FC9DE3C2FC7DE342FC5DE942F28
:103310004C2E5D2E21964AC1A2C1423409F075C0DF
:1033200060DE442311F041E09AC15BDE413410F0CD
:1033300042E095C1642E742E54DEB42EBB27A0E665
:1033400050DE4D936A94E1F7BB27A0E621E0A22E60
:103350004B2D463449F0453411F043E080C14D9186
:10336000DCDE7A94E1F77EC1E5E4FBE1EE0FFF1FBE
:1033700050DE08F423C030E475DE3D918DDE38E484
:10338000832F70DE3D91932F4C2E5D2E85DE21968E
:103390007A9431F07A9421F0AA2069F38A9459F74B
:1033A000AA2009F45FC18A943CE476DE352D74DEF0
:1033B000342D72DE30E070DE8C2C23C15523DAF020
:1033C0009D919F3F41F030E4832F4CDE392F64DE26
:1033D0004C2E5D2EF2D07A949D919F3F41F038E4BF
:1033E000832F40DE392F58DE4C2E5D2EE6D02196FD
:1033F0007A9421F737C13D2FA7DE32604DDE3C2F96
:103400004BDE3D91932F48DEEFCF4235E1F455235B
:1034100022F038E241DE3D2F03C03D2F95DE3160C2
:103420003BDE3C2F39DE37DE432FDFDD55234AF00C
:1034300030E232DE3D2F30DE3C2F2EDE2CDE432FFD
:10344000D4DD2196A3CE4736B9F4CBDDB42FC9DD48
:10345000A42FC7DD463439F0453409F000C147DEFA
:103460001197E9F793CE27DE55231AF01297D9F773
:103470008DCE1197C1F78ACE413429F4B2DDD42F15
:10348000B0DDC42FEFC0443419F4ABDD46DEEAC032
:10349000443611F42CDE7ACE4C3421F488DD82DD02
:1034A000C39AE0C0453409F4F9CF453669F43CEAE3
:1034B000F3DD552312F030E8EFDD34E0EDDD30E0F0
:1034C000EBDD08E2C6DDCEC04C3649F48ADD3CEACD
:1034D000E3DD552382F0342F306EDEDD07C0463643
:1034E00099F47FDD3CEAD8DD30EAD6DD3327D4DD40
:1034F000342FD2DD06C0342F307E3760CDDD30E092
:10350000CBDD0AE0A6DDAEC0433771F455235AF097
:1035100020E3122E222422E0322EB3DD3A94B1DDD4
:103520003324AFDD33CE9BC04D3649F43CE4B4DDEB
:10353000352DB2DD342DB0DD30E0AEDD62C04A3372
:1035400051F44FDD142E4DDD242E4BDD342E99DD4C
:1035500002E37FDD87C04E3269F443DD142E41DD86
:10356000242E3FDD342E3DDD83DD472F3EDD02E39B
:1035700070DD78C0423711F438E503C0463421F4D9
:1035800030E58ADD33270AC04E3419F438E584DD8E
:1035900004C0413551F430E57FDD38E07DDD33276F
:1035A0007BDD79DD432F21DDF1CD59C0E5E4FBE181
:1035B000EE0FFF1F2EDD18F055C021E0922EDD200A
:1035C000D1F09D15C1F08F7080622227552322F023
:1035D000382F62DD352D03C0352DB6DD31605CDD61
:1035E000342D5ADD58DD552312F430789078391790
:1035F00021F02A9559F70AE02CDD992099F19924B8
:103600000895513499F05332D1F09F3F79F08F7083
:1036100080622227382F40DD352D3EDD342D3CDD04
:103620003ADD391729F02A9509F0F4CF02E311DDCC
:10363000AA2019F0772009F09ECEAA2413C080EFAB
:103640002227522E382F28DD352D26DD342D24DD7E
:1036500022DD317069F32A9549F3F4CFC6DC4FE3DC
:10366000C4DC94CD4DE0C1DC91CD1300207F287FD8
:1036700030FF34FF387F48FF4CFF51FF55FF56FFA6
:1036800068FF6CFF86FF87FF000001400440054093
:1036900006400740084009400E101A100F201B205A
:1036A00014201C201D40231031203320354037408A
:1036B00039403D403E4057103A203B204140434076
:1036C0004440454046405E10604061406240634077
:1036D0006440664069206A207240734074407540BF
:1036E000762077207840794000003338000032326D
:1036F000000041565220495350005665722E332E19
:1037000038622028415652313039204D6F64652C83
:103710002050617274206F662049736F4A7461672C
:103720004953507777772E666C6F70707973706F2E
:103730006E67656F6E6C696E652E636F6D202620F7
:103740007777772E6D696B726F636F6E74726F6CC3
:103750006C65722D70726F6A656B74652E6465009E
:1037A000033089F0053089F0073089F00B3089F05B
:1037B0000F3089F0073189F00F3189F00F3289F02D
:1037C0000F3589F011C003E00FC005E00DC007E020
:1037D0000BC00BE009C00FE007C007E105C00FE117
:0E37E00003C00FE201C00FE510BD09B9089546
:0238000001C005
:10380400C0E5D4E0DEBFCDBF11241A8219821D8227
:103814001C821F821E821886F89481E080935500D2
:1038240082E080935500809134008F7B8093340034
:1038340080913500806480933500809137008860E2
:10384400809337000E940C1F80914E00816080930A
:103854004E0080914E00846080934E0010924D0083
:1038640010924C001A86198689859A8528E2843834
:10387400920741F48091380098E0892780933800BA
:103884001A86198689859A8501969A8789878091EF
:103894003300992780749070009799F480913800D0
:1038A40088608093380081E0809355001092550021
:1038B40010924E00809135008F7B809335000E94DA
:1038C400C71780912B0088233CF480912C008B87B0
:1038D4008B85833509F432C080914C0090914D0062
:1038E4003CE8803A930708F4BFCF8885813019F00B
:1038F40081E08887B9CF8091380088608093380050
:1039040081E0809355001092550010924E008091F2
:103914003300992780749070009741F080913500AE
:103924008F7B809335000E941C1F9ECF80913500B1
:103934008F7B809335000E94C71796CF8091380003
:1039440088608093380010924E000E94B41E0E943A
:10395400D01E8B838B81282F33273F872E878E851C
:103964009F858635910509F4B1C02E853F8527359D
:1039740031050CF04DC08E859F858534910509F481
:10398400D7C12E853F8526343105ECF48E859F857D
:103994008B31910509F4D9C12E853F852C31310530
:1039A4002CF48E859F85009791F2D8C12E853F8592
:1039B4002134310509F497C08E859F8583349105A0
:1039C40009F41DC1CBC12E853F852235310509F48B
:1039D400D7C08E859F85833591056CF42E853F85F0
:1039E4002C34310509F4A0C08E859F85803591055E
:1039F40009F496C0B3C12E853F852335310509F4FA
:103A04005BC08E859F858435910509F466C0A6C187
:103A14002E853F852D36310509F423C18E859F857A
:103A24008E369105F4F42E853F852336310509F44D
:103A3400D8C08E859F858436910534F42E853F85C4
:103A440021363105A9F18AC18E859F858436910579
:103A540009F478C02E853F852536310509F422C145
:103A64007DC18E859F858437910549F12E853F85DB
:103A74002537310564F48E859F8580379105A1F043
:103A84002E853F852337310509F452C067C18E85E1
:103A94009F858837910509F435C12E853F852937DF
:103AA400310509F43AC15AC183E50E94ED1E4FCF96
:103AB40089E50E94ED1E4BCF0E94B41E48CF84E7D7
:103AC4000E94ED1E80E00E94ED1E41CF81E30E9422
:103AD400ED1E80E30E94ED1E3ACF0E94D01E8DE0C1
:103AE4000E94ED1E34CF0E94D01E9927182F002764
:103AF4000E94D01E9927802B912B90932A018093AA
:103B040029012091290130912A01C901820F931FB3
:103B140090932D0180932C018DE00E94ED1E17CF10
:103B24008DE00E94ED1E13CF8DE00E94ED1E0FCF9D
:103B340082E00E94ED1E84E90E94ED1E8EE10E9447
:103B4400ED1E05CF8091290180933E0080912901CB
:103B540090912A01892F992780933F0080913C00FE
:103B6400992782709070009709F0F8CF80913C00FB
:103B7400816080933C0080913D000E94ED1EE7CE61
:103B840080915700992781709070009709F0F8CFC1
:103B940081E180935700E89580912C0190912D014B
:103BA40001969D878C87EC85FD8584918B878B8519
:103BB4000E94ED1E80912C0190912D019D878C8790
:103BC400EC85FD8584918B878B850E94ED1E809109
:103BD4002C0190912D01029690932D0180932C013C
:103BE400B6CE80913800877F809338000E94D01E23
:103BF40099279A8389838DE00E94ED1EA8CE0E94A6
:103C0400D01E9927382F222789819A81822B932BC2
:103C14009A838983809138008860809338008091EA
:103C24005700992781709070009709F0F8CF41E010
:103C340020912C0130912D0189819A810C01F90187
:103C440040935700E895112480912C0190912D0107
:103C5400029690932D0180932C018DE00E94ED1E1D
:103C640076CE8091290190912A0137E1803893071B
:103C740020F08DE00E94ED1E6ACE809157009927B6
:103C840081709070009709F0F8CF25E080912C01A5
:103C940090912D01FC0120935700E8958DE00E943E
:103CA400ED1E55CE10922A0110922901809129010E
:103CB40090912A0127E181309207E0F423E080917A
:103CC400290190912A01FC0120935700E8958091E5
:103CD4005700992781709070009709F0F8CF809170
:103CE400290190912A0180589F4F90932A01809333
:103CF4002901DCCF81E180935700E8958DE00E9493
:103D0400ED1E25CE0E94D01E80913800877F8093BF
:103D140038008DE00E94ED1E1ACE0E94D01E8091C4
:103D240038008860809338008DE00E94ED1E0FCE2D
:103D340088E190E028E00FB6F894A89581BD0FBE05
:103D440021BD8DE00E94ED1E02CE10922D01109235
:103D54002C0110922A0110922901F9CD8FE30E94BF
:103D6400ED1EF5CDCF93DF93CDB7DEB781E40E948E
:103D7400ED1E86E50E94ED1E82E50E94ED1E82E4A2
:103D84000E94ED1E8FE40E94ED1E8FE40E94ED1E42
:103D940084E50E94ED1EDF91CF910895CF93DF93C8
:103DA400CDB7DEB721970FB6F894DEBF0FBECDBFF7
:103DB40080912B0088230CF0FBCF80912C00898309
:103DC4008981992721960FB6F894DEBF0FBECDBF27
:103DD400DF91CF910895CF93DF93CDB7DEB72197CD
:103DE4000FB6F894DEBF0FBECDBF898380912B0040
:103DF400992780729070009709F4F8CF8981809395
:103E04002C0021960FB6F894DEBF0FBECDBFDF9114
:103E1400CF910895CF93DF93CDB7DEB787E1809339
:103E2400290088E180932A0086E880934000DF918E
:103E3400CF910895CF93DF93CDB7DEB7F0E0E0E004
:083E44000994DF91CF9108956C
:0400000300002F00CA
:00000001FF
